:020000040000FA
:02000000ED28E9
:08000800A000030EA10083011A
:100010002D0882078629B82A210E8300A00E200E03
:10002000090082073F3406345B344F3466346D3444
:100030007D3407347F34673482070134023404345A
:100040000834820703340334033403349434A5346E
:10005000C634D734E834F9348207013401348434A7
:10006000843484349534A634B734C834D934820700
:10007000AA343734113405342908A90A82076434B4
:100080000534AD34023452340134A13400344E34DA
:100090000034213400341434003405340034290889
:1000A000A90A8207733450345C347C3473343E3490
:1000B00038346D343E345C34383438343E345C3457
:1000C000383476345E3404345C345E343834793415
:1000D0005E346D347134503479346F3400343934D3
:1000E00054347834003439347734733439345C34EC
:1000F0000434383400346D3406343D3454347834A8
:100100006D34393400346D3479345034153404345A
:100110005E34043450345234D8345C345034523465
:10012000D8340434083437340834373454345C3425
:1001300004346D34043450344F347F3473342A34EF
:10014000153400346D3478343F3473340034003463
:1001500000346D34003400346D343F3400346D3479
:100160003F343F3400340034ED343F3406345B34E4
:100170003F343F345B3466343F343F3466347F343D
:100180003F343F3467347D343F343F3400340634E9
:10019000E7345B3400344F34FF34663400346D345C
:1001A00087347D3406340634ED345B3436088207F8
:1001B000B82BFD2A112C0F2C052C092C722C3C2C51
:1001C0005E2B902B2F2BF82C1B2E562E0A2A4C2AF6
:1001D000C62AEB29C7299329B82E83163F308500FC
:1001E00000308600B03087008830810083120430F0
:1001F0009200D0015014CC0149217321E830B300A2
:100200000330B4003030B5003B218B133608662133
:100210008A250530E724071A1B29871E08298A2505
:100220000530E724071A2829871A0F29B603133047
:10023000B61BB60005298A250530E724871A282928
:10024000071A1B29B60A3608143A0319B6010529FC
:100250003B212B21D6288316051485140516051578
:10026000871707178515851606309F00831208002B
:10027000231D08002311BB01BC0136080526BC0A5A
:100280003A080526BC0A39080526BC0A380805269E
:100290000800BB01BC01F725B6003608EC3E031888
:1002A000B601BC0AF725BA003A08FC3E0318BA01A9
:1002B000BC0AF725B900F13E0318B901BC0AF725BD
:1002C000B8003808FC3E0318B8010800A900031064
:1002D000A90DA90D4F20C8004F20C9004F20CA000A
:1002E0004F20CB0008002B30FE230030C8007C21BB
:1002F000360866217C2108001E30A9008A250530B9
:10030000E724A40B7E29A90B7E2908000B11231ECC
:100310008E29231205102C0881000C2823160514A1
:100320002B0881000C28831605108230810083126F
:100330000030AD008B168B173508023EFE233508C2
:10034000003CAB003508603C003CAC000530E724C5
:100350008A250530E7248A25B00BA6291930B0007C
:100360000530E7248A25071EB929871EBF29B00159
:10037000B029871E0529B50BB503B50A9C29071EB0
:100380000529B50A3508603A0319B5039C29831677
:1003900005108312D8210530A4008A250530E724F2
:1003A000A40BCD29B323071ACA29871ACA290529FC
:1003B0002630A40005141430D100D10BDD29000033
:1003C0000000000005101430D100D10BE529000019
:1003D000A40BDA2908008316051083125530BD00DE
:1003E000FF213D1805143D1C05108A254130D10020
:1003F000D10BF829871AF029071AF02905293D0899
:100400003E07BE003F07BF000310BD0C0318BD1719
:10041000BD070800831605108312DC30B0000530DC
:10042000B1003008C0003108C100C201C301D625A7
:10043000A7253230A4008A250A30E724A40B1B2A02
:100440003008BC003108BB00B3234122071E362A06
:10045000871E2B2A192A071E05290A30B007031800
:10046000B10A3108093A0319382A112A871E0529C9
:10047000F630B007031CB1033108023A03192D2AE4
:10048000112ABB0ABC0A051400000000BC0B442A58
:10049000BB0B462A0510080083168516871705151D
:1004A0008511051406309F0083128511E923051874
:1004B000A02A8A25071EA02A871EA02A051C592AC1
:1004C000C001C101C201C301000000000000702A88
:1004D0000000000000000330A2008A25A20B6E2A53
:1004E000051C7A2A0A30C007031C682AC10F692A32
:1004F000C20F6A2AC401C501C601C70100000B3042
:10050000A200882A0000000000000330A2008A2513
:10051000A20B882A0518942A0A30C407031C822AD1
:10052000C50F832AC60F842A231F9C2A6924D62537
:10053000A725A7248A25A02AD625A725A7248A256A
:10054000071AAB2A2313C801C901CA017630CB00B0
:100550008A25871E0529871A562A2317C801C9012B
:10056000CA013830CB008A25071E0529562A080003
:100570000B113308B00734080318340FB107B11F4B
:100580000510B11B0514B73081070C288316051020
:100590008830810083120130AD008B178B16330831
:1005A000C0003408C100C201C301D625A725370801
:1005B000A4008A250530E724A40BD92AFB30B7070D
:1005C0003708FB3E0318E62A0630B700071EF22A5A
:1005D000871EEC2AB701D72A071E0529B30A03197B
:1005E000B40ACF2A871E0529FF30B307031CB403C2
:1005F000B41FCF2AB301B401CF2A831606309F005F
:1006000083123A08153E66213A083720B0000F2BB6
:10061000831605100000051483124817162B0514C5
:10062000051A0510083005180130C8003008DD240F
:100630000230DD24071A1F2B871A082B0429871A7A
:100640000F2B0530E724F9238A25071E0429871E6E
:10065000212BBA0A3A08033C031CBA01012B83166A
:100660008713851106309F00831287138511C801F7
:1006700005301120C90000301120CA00CB00301F06
:10068000481785154D23B00A301B481385114D239B
:10069000071A432B871A3F2B05292030A4008A25EF
:1006A0000E305523A40B4F2B0800D1000000000092
:1006B000000000000000D10B562B080083168511A6
:1006C0008312851505102314B323C001C101C20193
:1006D000C30183160514831200000000000000000F
:1006E000000000000000000000000000000000000A
:1006F0000000000000000518852BC00F722BC10FF1
:10070000722BC20F722BC30F722B8316051083122C
:10071000D625F124E923071A8A2B871A642B052989
:1007200083168510831285102314B3235030E724D9
:10073000C001C101C201C30185140000051CA82B22
:10074000C00F9D2BC10F9D2BC20F9D2BC30F9D2B47
:100750008510D6250330A525CA17E923071AAD2B26
:10076000871A952B05290710871007118711080094
:10077000831687130713A83081000E309F00831261
:100780008717071381309F00CD01FF308100071AC2
:10079000CC2B871ACC2B052930243B08283C031886
:1007A000D92B3B08B43C031CD72B4030DA2B7630D6
:1007B000DA2B3830F7230B1DE32B0B11FF308100B0
:1007C000B0017330C900EB23B00AB0080319C901A6
:1007D000C72BA401F02BA401A417F02BA40124170C
:1007E0008A25A7240530E724A40BF02B0800C800B5
:1007F000FA2BC801C901CA01CB010800C000C10120
:10080000C201C301D625A7250800A31283168713AA
:10081000122CA3128316851283128516122CA3168E
:10082000122CA31283168E309F00831287178130FB
:100830009F00302411273C08C0003B08C100C201C2
:10084000C301D625A725C917C830A4008A250530BD
:10085000E724A40B262C071A192C871A192C052912
:100860001F15000000001F19332C83161E08831269
:10087000BC001E08BB0008008316851687130515EB
:1008800085150514A830810006309F008312871754
:100890008101C401C501C601C7016924D625033001
:1008A000A5258A255E24071E582C871E482C4D2C12
:1008B000871E05296924D6250730502C0108C4005D
:1008C0000B1D08000B11C50F0800C60F0800C70A52
:1008D00008004408C0004508C1004608C200470897
:1008E000C3000800831685168717051585110514A2
:1008F000A730810006309F0083120511C001C1019D
:10090000C201C301D625A725071A8A2C871E0529EF
:100910000330A5258E24B7249824822C85128101CA
:10092000C001C101C201C3018316851683120800EC
:1009300085128316851283120108C100C001C0030D
:10094000851685120108410603199F2C08004D0EDB
:100950000339483E8400CD1B8017CE0A0319CF0A05
:10096000CF1EB52C4D1B8013080000000800EE3090
:10097000B000A730B10000000000CB248A25A724D6
:10098000D224B00BBB2CB10BBD2C0830B000D2244C
:10099000B00BC72C08001030A900A90BCD2C00000B
:1009A000000008000B1DD92C0B11C20A0319C30A41
:1009B00008000000000000000800D200D300530827
:1009C000D1008A25D10BE12CD20BDF2C0800D300FB
:1009D000D200D100D10BEA2CD20BE92CD30BE82C9E
:1009E0000800BB2524082C20CD000F39A400AD2D14
:1009F0008316051185108510831285100711871144
:100A0000BF30860025252830A40000004C25A40B0B
:100A1000052D0F30A4005525542554254B254B2575
:100A20004B254B254B254B254B254B254B254B2546
:100A30000000A40B0B2D1130A4004C250000A40BCA
:100A40001D2D4125871A022D05290630A400051108
:100A5000732505152E307A25A40B272D0630A4000A
:100A600005112E307A2505157525A40B302D06307D
:100A7000A4000511732505152E307A25A40B392DF8
:100A80000800792505116D25762505157E25593037
:100A90007A2500000800792505116D2576250515B4
:100AA0005D307A2500000800792505116D25762531
:100AB00005156B256B251330A90000000000000010
:100AC000000000000000851400008510A90B5D2DBA
:100AD00005307A250800000000000000000000003A
:100AE0000000000000000000000000000000000006
:100AF00000000800A900A90B7B2D0800DB0A0710E5
:100B000087105B1C07145B18871400000800F03086
:100B100087050800F03087054C08483E840000082F
:100B20005005FF3A86004C081C2087040310D00DA6
:100B30000318A02D000000000000000000000800C5
:100B40005014CC0A4C19CC010800A400AD2DBB25D3
:100B500024082120CD000F39A400B625C800B625F1
:100B6000C900B625CA00B625CB0008002408A40396
:100B7000C525112008000930A4002408C525003A25
:100B8000031D0800A40BBD2D0800A9000301A91B2B
:100B900008000310A90C2908A90D543E8400000880
:100BA000A7002918A70E27080F3908002030DA00FF
:100BB000D401D501D601D701D801543084000530C5
:100BC000D900333080078019F039801B0F3980023B
:100BD000840AD90BE12DC00DC10DC20DC30DD40D7A
:100BE000D50DD60DD70DD80DDA0BDD2D08008312EB
:100BF00003173C088D003B088F0083168C130C14E0
:100C000083120C08031383120800831203178C004D
:100C10003C088D003B088F0083168C130C15553053
:100C20008D00AA308D008C14000000008C18162E48
:100C300083120313080087258316051483123808CE
:100C4000A9000310A90D3C20AE003C20AF001930D4
:100C5000380766218A25871E482E071A2A2E871EE6
:100C600005298A264130A8001A30A50028089126B7
:100C7000A80A2B30DD24A50B362E0D3091266430CA
:100C8000DD240A309126DC30DD24071E2A2E1B2E9F
:100C900087251430E724071E0529871E482EB80A29
:100CA0003808083A0319B80123151B2E3908013EEC
:100CB000FE233930C8007630C9008316051483122C
:100CC0008A25871E7F2E071A602E8A262D30AE00B9
:100CD000AF013908903891263C3091262830912672
:100CE0001430DD24071E702E3908903891263C30D0
:100CF0009126003091263821FA30DD24562E6430BA
:100D0000DD24071E0529871E7F2E2315B90A0F3003
:100D1000B905562EA310051CA314831605108312C3
:100D20000800A401A415A700A326AD262718A8260D
:100D3000271CA326A70CA40B952EAD26A826AD260E
:100D4000AD26AD260034A31C0510A31805140034ED
:100D5000A31C0514A318051000342F08AA002E08A0
:100D6000A900AA0AA90AA90BB32EAA0BB32E003414
:100D700083168713831287130130900087250C2771
:100D8000F926F126FD26F126031DD52E071ACB2EB6
:100D9000871ACE2E0529871AC22EBE2EDF26DF2601
:100DA000DF26DF26DF26071ED22EDF26F126031DD3
:100DB000DB2E071AD52EFD26871ADB2EBE2EFD262A
:100DC0000C1CDF2E87250C1000308E0000308F00A9
:100DD000F92600275C08FC3E031CC9170319CA1733
:100DE00000345D08A9000508DD0029060139031952
:100DF00000346924D625A72500348A250530E72C40
:100E0000C40A031D0034C50A031D0034C60A031DAD
:100E10000034C70A031D0034C401C501C601C7015F
:100E20000034A31A182F0130C000F430C1001C2F69
:100E30000930C000C430C10027270330BB00FF3099
:100E4000BC00CC274208BB004308BC000800C4011A
:100E5000C5013B0803104018C407C40CC50CC018DA
:100E6000C407C40CC50C4019C407C40CC50CC01978
:100E7000C407C40CC50C401AC407C40CC50CC01A66
:100E8000C407C40CC50C401BC407C40CC50CC01B54
:100E9000C407C40CC50CC201C3013C0803104118AF
:100EA000C207C20CC30CC118C207C20CC30C411943
:100EB000C207C20CC30CC119C207C20CC30C411A31
:100EC000C207C20CC30CC11AC207C20CC30C411B1F
:100ED000C207C20CC30CC11BC207C20CC30CC601A3
:100EE000C7013B0803104118C607C60CC70CC11840
:100EF000C607C60CC70C4119C607C60CC70CC119DA
:100F0000C607C60CC70C411AC607C60CC70CC11AC7
:100F1000C607C60CC70C411BC607C60CC70CC11BB5
:100F2000C607C60CC70C4708C20746080318460F79
:100F3000C5070318C40AC601C7013C0803104018BE
:100F4000C607C60CC70CC018C607C60CC70C40198C
:100F5000C607C60CC70CC019C607C60CC70C401A7A
:100F6000C607C60CC70CC01AC607C60CC70C401B68
:100F7000C607C60CC70CC01BC607C60CC70C470863
:100F8000C20746080318460FC5070318C40A4508D8
:100F9000C1004408C00008002030A200C401C501FF
:100FA0000310C30DC20DC10DC00DC50DC40D031836
:100FB000E12F3B084402031DDF2F3C084502031CC0
:100FC000E82F3C08C502031CC4033B08C4024314B9
:060FD000A20BD02F080067
:02400E00323F3F
:00000001FF
